 management

 Timestamp is 029a345f (reproducible build file hash)

 Preferred load address is 10000000

 Start         Length     Name                   Class
 0001:00000000 0000156bH .text$mn                CODE
 0002:00000000 0000008cH .idata$5                DATA
 0002:0000008c 00000008H .00cfg                  DATA
 0002:00000094 00000004H .CRT$XCA                DATA
 0002:00000098 00000004H .CRT$XCZ                DATA
 0002:0000009c 00000004H .CRT$XIA                DATA
 0002:000000a0 00000004H .CRT$XIZ                DATA
 0002:000000a4 00000004H .CRT$XPA                DATA
 0002:000000a8 00000004H .CRT$XPZ                DATA
 0002:000000ac 00000004H .CRT$XTA                DATA
 0002:000000b0 00000008H .CRT$XTZ                DATA
 0002:000000b4 00000000H .gfids$y                DATA
 0002:000000b8 000002c8H .rdata                  DATA
 0002:00000380 00000000H .rdata$CastGuardVftablesA DATA
 0002:00000380 00000000H .rdata$CastGuardVftablesC DATA
 0002:00000380 00000004H .rdata$sxdata           DATA
 0002:00000384 00000064H .rdata$voltmd           DATA
 0002:000003e8 000002a0H .rdata$zzzdbg           DATA
 0002:00000688 00000004H .rtc$IAA                DATA
 0002:0000068c 00000004H .rtc$IZZ                DATA
 0002:00000690 00000004H .rtc$TAA                DATA
 0002:00000694 00000004H .rtc$TZZ                DATA
 0002:00000698 00000088H .xdata$x                DATA
 0002:00000720 00001218H .edata                  DATA
 0002:00001938 00000078H .idata$2                DATA
 0002:000019b0 00000014H .idata$3                DATA
 0002:000019c4 0000008cH .idata$4                DATA
 0002:00001a50 0000031eH .idata$6                DATA
 0003:00000000 00000018H .data                   DATA
 0003:00000018 0000037cH .bss                    DATA
 0004:00000000 00000060H .rsrc$01                DATA
 0004:00000060 00000338H .rsrc$02                DATA

  Address         Publics by Value              Rva+Base       Lib:Object

 0000:00000000       ___AbsoluteZero            00000000     <absolute>
 0000:00000000       ___arm64x_extra_rfe_table  00000000     <absolute>
 0000:00000000       ___arm64x_extra_rfe_table_size 00000000     <absolute>
 0000:00000000       ___arm64x_native_entrypoint 00000000     <absolute>
 0000:00000000       ___arm64x_redirection_metadata 00000000     <absolute>
 0000:00000000       ___arm64x_redirection_metadata_count 00000000     <absolute>
 0000:00000000       ___dynamic_value_reloc_table 00000000     <absolute>
 0000:00000000       ___enclave_config          00000000     <absolute>
 0000:00000000       ___guard_check_icall_a64n_fptr 00000000     <absolute>
 0000:00000000       ___guard_eh_cont_count     00000000     <absolute>
 0000:00000000       ___guard_eh_cont_table     00000000     <absolute>
 0000:00000000       ___guard_fids_count        00000000     <absolute>
 0000:00000000       ___guard_fids_table        00000000     <absolute>
 0000:00000000       ___guard_iat_count         00000000     <absolute>
 0000:00000000       ___guard_iat_table         00000000     <absolute>
 0000:00000000       ___guard_longjmp_count     00000000     <absolute>
 0000:00000000       ___guard_longjmp_table     00000000     <absolute>
 0000:00000000       ___hybrid_auxiliary_delayload_iat 00000000     <absolute>
 0000:00000000       ___hybrid_auxiliary_delayload_iat_copy 00000000     <absolute>
 0000:00000000       ___hybrid_auxiliary_iat    00000000     <absolute>
 0000:00000000       ___hybrid_auxiliary_iat_copy 00000000     <absolute>
 0000:00000000       ___hybrid_code_map         00000000     <absolute>
 0000:00000000       ___hybrid_code_map_count   00000000     <absolute>
 0000:00000000       ___hybrid_image_info_bitfield 00000000     <absolute>
 0000:00000000       ___x64_code_ranges_to_entry_points 00000000     <absolute>
 0000:00000000       ___x64_code_ranges_to_entry_points_count 00000000     <absolute>
 0000:00000001       ___safe_se_handler_count   00000001     <absolute>
 0000:00000100       ___guard_flags             00000100     <absolute>
 0000:00000000       ___ImageBase               10000000     <linker-defined>
 0001:00000000       _Java_sun_management_ClassLoadingImpl_setVerboseClass@12 10001000 f   ClassLoadingImpl.obj
 0001:00000015       _Java_sun_management_GarbageCollectorImpl_getCollectionCount@8 10001015 f   GarbageCollectorImpl.obj
 0001:0000002a       _Java_sun_management_GarbageCollectorImpl_getCollectionTime@8 1000102a f   GarbageCollectorImpl.obj
 0001:0000003f       _Java_sun_management_HotspotThread_getInternalThreadCount@8 1000103f f   HotspotThread.obj
 0001:00000052       _Java_sun_management_HotspotThread_getInternalThreadTimes0@16 10001052 f   HotspotThread.obj
 0001:00000069       _Java_sun_management_MemoryImpl_getMemoryManagers0@8 10001069 f   MemoryImpl.obj
 0001:0000007a       _Java_sun_management_MemoryImpl_getMemoryPools0@8 1000107a f   MemoryImpl.obj
 0001:0000008b       _Java_sun_management_MemoryImpl_getMemoryUsage0@12 1000108b f   MemoryImpl.obj
 0001:0000009e       _Java_sun_management_MemoryImpl_setVerboseGC@12 1000109e f   MemoryImpl.obj
 0001:000000b3       _Java_sun_management_MemoryManagerImpl_getMemoryPools0@8 100010b3 f   MemoryManagerImpl.obj
 0001:000000de       _Java_sun_management_MemoryPoolImpl_getCollectionUsage0@8 100010de f   MemoryPoolImpl.obj
 0001:000000e6       _Java_sun_management_MemoryPoolImpl_getMemoryManagers0@8 100010e6 f   MemoryPoolImpl.obj
 0001:00000111       _Java_sun_management_MemoryPoolImpl_getPeakUsage0@8 10001111 f   MemoryPoolImpl.obj
 0001:0000013c       _Java_sun_management_MemoryPoolImpl_getUsage0@8 1000113c f   MemoryPoolImpl.obj
 0001:00000167       _Java_sun_management_MemoryPoolImpl_resetPeakUsage0@8 10001167 f   MemoryPoolImpl.obj
 0001:00000186       _Java_sun_management_MemoryPoolImpl_setCollectionThreshold0@24 10001186 f   MemoryPoolImpl.obj
 0001:000001eb       _Java_sun_management_MemoryPoolImpl_setPoolCollectionSensor@12 100011eb f   MemoryPoolImpl.obj
 0001:00000207       _Java_sun_management_MemoryPoolImpl_setPoolUsageSensor@12 10001207 f   MemoryPoolImpl.obj
 0001:00000223       _Java_sun_management_MemoryPoolImpl_setUsageThreshold0@24 10001223 f   MemoryPoolImpl.obj
 0001:00000288       _Java_sun_management_ThreadImpl_dumpThreads0@24 10001288 f   ThreadImpl.obj
 0001:000002a9       _Java_sun_management_ThreadImpl_findDeadlockedThreads0@8 100012a9 f   ThreadImpl.obj
 0001:000002ba       _Java_sun_management_ThreadImpl_findMonitorDeadlockedThreads0@8 100012ba f   ThreadImpl.obj
 0001:000002c9       _Java_sun_management_ThreadImpl_getThreadAllocatedMemory0@16 100012c9 f   ThreadImpl.obj
 0001:000002e0       _Java_sun_management_ThreadImpl_getThreadAllocatedMemory1@16 100012e0 f   ThreadImpl.obj
 0001:000002f7       _Java_sun_management_ThreadImpl_getThreadInfo1@20 100012f7 f   ThreadImpl.obj
 0001:00000312       _Java_sun_management_ThreadImpl_getThreadTotalCpuTime0@16 10001312 f   ThreadImpl.obj
 0001:0000032b       _Java_sun_management_ThreadImpl_getThreadTotalCpuTime1@16 1000132b f   ThreadImpl.obj
 0001:00000344       _Java_sun_management_ThreadImpl_getThreadUserCpuTime0@16 10001344 f   ThreadImpl.obj
 0001:0000035d       _Java_sun_management_ThreadImpl_getThreadUserCpuTime1@16 1000135d f   ThreadImpl.obj
 0001:00000376       _Java_sun_management_ThreadImpl_getThreads@8 10001376 f   ThreadImpl.obj
 0001:0000037b       _Java_sun_management_ThreadImpl_getTotalThreadAllocatedMemory@8 1000137b f   ThreadImpl.obj
 0001:0000038d       _Java_sun_management_ThreadImpl_resetContentionTimes0@16 1000138d f   ThreadImpl.obj
 0001:000003a9       _Java_sun_management_ThreadImpl_resetPeakThreadCount0@8 100013a9 f   ThreadImpl.obj
 0001:000003c7       _Java_sun_management_ThreadImpl_setThreadAllocatedMemoryEnabled0@12 100013c7 f   ThreadImpl.obj
 0001:000003dc       _Java_sun_management_ThreadImpl_setThreadContentionMonitoringEnabled0@12 100013dc f   ThreadImpl.obj
 0001:000003f1       _Java_sun_management_ThreadImpl_setThreadCpuTimeEnabled0@12 100013f1 f   ThreadImpl.obj
 0001:00000406       _Java_sun_management_VMManagementImpl_getAvailableProcessors@8 10001406 f   VMManagementImpl.obj
 0001:0000040e       _Java_sun_management_VMManagementImpl_getClassInitializationTime@8 1000140e f   VMManagementImpl.obj
 0001:00000421       _Java_sun_management_VMManagementImpl_getClassLoadingTime@8 10001421 f   VMManagementImpl.obj
 0001:00000434       _Java_sun_management_VMManagementImpl_getClassVerificationTime@8 10001434 f   VMManagementImpl.obj
 0001:00000447       _Java_sun_management_VMManagementImpl_getDaemonThreadCount@8 10001447 f   VMManagementImpl.obj
 0001:0000045a       _Java_sun_management_VMManagementImpl_getInitializedClassCount@8 1000145a f   VMManagementImpl.obj
 0001:0000046d       _Java_sun_management_VMManagementImpl_getLiveThreadCount@8 1000146d f   VMManagementImpl.obj
 0001:00000480       _Java_sun_management_VMManagementImpl_getLoadedClassSize@8 10001480 f   VMManagementImpl.obj
 0001:00000493       _Java_sun_management_VMManagementImpl_getMethodDataSize@8 10001493 f   VMManagementImpl.obj
 0001:000004a6       _Java_sun_management_VMManagementImpl_getPeakThreadCount@8 100014a6 f   VMManagementImpl.obj
 0001:000004b9       _Java_sun_management_VMManagementImpl_getProcessId@8 100014b9 f   VMManagementImpl.obj
 0001:000004cf       _Java_sun_management_VMManagementImpl_getSafepointCount@8 100014cf f   VMManagementImpl.obj
 0001:000004e2       _Java_sun_management_VMManagementImpl_getSafepointSyncTime@8 100014e2 f   VMManagementImpl.obj
 0001:000004f5       _Java_sun_management_VMManagementImpl_getStartupTime@8 100014f5 f   VMManagementImpl.obj
 0001:00000508       _Java_sun_management_VMManagementImpl_getTotalApplicationNonStoppedTime@8 10001508 f   VMManagementImpl.obj
 0001:0000051b       _Java_sun_management_VMManagementImpl_getTotalClassCount@8 1000151b f   VMManagementImpl.obj
 0001:0000052e       _Java_sun_management_VMManagementImpl_getTotalCompileTime@8 1000152e f   VMManagementImpl.obj
 0001:00000541       _Java_sun_management_VMManagementImpl_getTotalSafepointTime@8 10001541 f   VMManagementImpl.obj
 0001:00000554       _Java_sun_management_VMManagementImpl_getTotalThreadCount@8 10001554 f   VMManagementImpl.obj
 0001:00000567       _Java_sun_management_VMManagementImpl_getUnloadedClassCount@8 10001567 f   VMManagementImpl.obj
 0001:0000057a       _Java_sun_management_VMManagementImpl_getUnloadedClassSize@8 1000157a f   VMManagementImpl.obj
 0001:0000058d       _Java_sun_management_VMManagementImpl_getUptime0@8 1000158d f   VMManagementImpl.obj
 0001:000005a0       _Java_sun_management_VMManagementImpl_getVerboseClass@8 100015a0 f   VMManagementImpl.obj
 0001:000005b1       _Java_sun_management_VMManagementImpl_getVerboseGC@8 100015b1 f   VMManagementImpl.obj
 0001:000005c2       _Java_sun_management_VMManagementImpl_getVersion0@8 100015c2 f   VMManagementImpl.obj
 0001:0000061a       _Java_sun_management_VMManagementImpl_getVmArguments0@8 1000161a f   VMManagementImpl.obj
 0001:00000626       _Java_sun_management_VMManagementImpl_initOptionalSupportFields@8 10001626 f   VMManagementImpl.obj
 0001:00000737       _Java_sun_management_VMManagementImpl_isThreadAllocatedMemoryEnabled@8 10001737 f   VMManagementImpl.obj
 0001:00000748       _Java_sun_management_VMManagementImpl_isThreadContentionMonitoringEnabled@8 10001748 f   VMManagementImpl.obj
 0001:00000759       _Java_sun_management_VMManagementImpl_isThreadCpuTimeEnabled@8 10001759 f   VMManagementImpl.obj
 0001:0000076a       ___local_stdio_printf_options 1000176a f i VMManagementImpl.obj
 0001:000007a2       _snprintf                  100017a2 f i VMManagementImpl.obj
 0001:000007bc       _vsnprintf                 100017bc f i VMManagementImpl.obj
 0001:000007ee       _JNI_OnLoad@8              100017ee f   management.obj
 0001:0000084c       _JVM_GetAllThreads@8       1000184c f   jvm:jvm.dll
 0001:00000852       _JVM_ActiveProcessorCount@0 10001852 f   jvm:jvm.dll
 0001:00000858       _JVM_GetVmArguments@4      10001858 f   jvm:jvm.dll
 0001:0000085e       _JVM_GetManagement@4       1000185e f   jvm:jvm.dll
 0001:00000864       _JNU_ThrowInternalError@8  10001864 f   java:java.dll
 0001:0000086a       @__security_check_cookie@4 1000186a f   MSVCRT:secchk.obj
 0001:00000bb8       __DllMainCRTStartup@12     10001bb8 f   MSVCRT:dll_dllmain.obj
 0001:00000bdb       ___raise_securityfailure   10001bdb f   MSVCRT:gs_report.obj
 0001:00000c03       ___report_gsfailure        10001c03 f   MSVCRT:gs_report.obj
 0001:00000d4a       ___security_init_cookie    10001d4a f   MSVCRT:gs_support.obj
 0001:00000d95       _DllMain@12                10001d95 f   MSVCRT:dll_dllmain_stub.obj
 0001:00000db7       ?__scrt_initialize_type_info@@YAXXZ 10001db7 f   MSVCRT:tncleanup.obj
 0001:00000dc3       ?__scrt_uninitialize_type_info@@YAXXZ 10001dc3 f   MSVCRT:tncleanup.obj
 0001:00000dcf       ___local_stdio_scanf_options 10001dcf f i MSVCRT:default_local_stdio_options.obj
 0001:00000dd5       ___scrt_initialize_default_local_stdio_options 10001dd5 f   MSVCRT:default_local_stdio_options.obj
 0001:00000e36       ___scrt_acquire_startup_lock 10001e36 f   MSVCRT:utility.obj
 0001:00000e68       ___scrt_dllmain_after_initialize_c 10001e68 f   MSVCRT:utility.obj
 0001:00000e93       ___scrt_dllmain_before_initialize_c 10001e93 f   MSVCRT:utility.obj
 0001:00000ea1       ___scrt_dllmain_crt_thread_attach 10001ea1 f   MSVCRT:utility.obj
 0001:00000ec0       ___scrt_dllmain_crt_thread_detach 10001ec0 f   MSVCRT:utility.obj
 0001:00000ecd       ___scrt_dllmain_exception_filter 10001ecd f   MSVCRT:utility.obj
 0001:00000f01       ___scrt_dllmain_uninitialize_c 10001f01 f   MSVCRT:utility.obj
 0001:00000f24       ___scrt_dllmain_uninitialize_critical 10001f24 f   MSVCRT:utility.obj
 0001:00000f31       ___scrt_initialize_crt     10001f31 f   MSVCRT:utility.obj
 0001:00000f6a       ___scrt_initialize_onexit_tables 10001f6a f   MSVCRT:utility.obj
 0001:00000ff1       ___scrt_is_nonwritable_in_current_image 10001ff1 f   MSVCRT:utility.obj
 0001:00001085       ___scrt_release_startup_lock 10002085 f   MSVCRT:utility.obj
 0001:000010a2       ___scrt_uninitialize_crt   100020a2 f   MSVCRT:utility.obj
 0001:000010ca       ___scrt_get_dyn_tls_init_callback 100020ca f   MSVCRT:dyn_tls_init.obj
 0001:000010d0       ___scrt_fastfail           100020d0 f   MSVCRT:utility_desktop.obj
 0001:000011eb       __crt_debugger_hook        100021eb f   MSVCRT:utility_desktop.obj
 0001:000011f3       __RTC_Initialize           100021f3 f   MSVCRT:initsect.obj
 0001:0000121f       __RTC_Terminate            1000221f f   MSVCRT:initsect.obj
 0001:00001250       __SEH_prolog4              10002250 f   MSVCRT:sehprolg4.obj
 0001:00001295       __except_handler4          10002295 f   MSVCRT:chandler4gs.obj
 0001:000012c4       @_guard_check_icall_nop@4  100022c4 f i MSVCRT:guard_support.obj
 0001:000012c7       ___isa_available_init      100022c7 f   MSVCRT:cpu_disp.obj
 0001:0000149b       __get_startup_argv_mode    1000249b f   MSVCRT:argv_mode.obj
 0001:0000149f       ___scrt_is_ucrt_dll_in_use 1000249f f   MSVCRT:ucrt_detection.obj
 0001:000014ab       ___std_type_info_destroy_list 100024ab f   vcruntime:VCRUNTIME140.dll
 0001:000014b1       _memset                    100024b1 f   vcruntime:VCRUNTIME140.dll
 0001:000014b7       __except_handler4_common   100024b7 f   vcruntime:VCRUNTIME140.dll
 0001:000014bd       __initterm                 100024bd f   ucrt:api-ms-win-crt-runtime-l1-1-0.dll
 0001:000014c3       __initterm_e               100024c3 f   ucrt:api-ms-win-crt-runtime-l1-1-0.dll
 0001:000014c9       __seh_filter_dll           100024c9 f   ucrt:api-ms-win-crt-runtime-l1-1-0.dll
 0001:000014cf       __configure_narrow_argv    100024cf f   ucrt:api-ms-win-crt-runtime-l1-1-0.dll
 0001:000014d5       __initialize_narrow_environment 100024d5 f   ucrt:api-ms-win-crt-runtime-l1-1-0.dll
 0001:000014db       __initialize_onexit_table  100024db f   ucrt:api-ms-win-crt-runtime-l1-1-0.dll
 0001:000014e1       __execute_onexit_table     100024e1 f   ucrt:api-ms-win-crt-runtime-l1-1-0.dll
 0001:000014e7       __cexit                    100024e7 f   ucrt:api-ms-win-crt-runtime-l1-1-0.dll
 0001:000014ed       ___acrt_initialize         100024ed f   MSVCRT:ucrt_stubs.obj
 0001:000014ed       ___acrt_thread_attach      100024ed f   MSVCRT:ucrt_stubs.obj
 0001:000014ed       ___acrt_thread_detach      100024ed f   MSVCRT:ucrt_stubs.obj
 0001:000014ed       ___acrt_uninitialize       100024ed f   MSVCRT:ucrt_stubs.obj
 0001:000014ed       ___acrt_uninitialize_critical 100024ed f   MSVCRT:ucrt_stubs.obj
 0001:000014ed       ___scrt_stub_for_acrt_initialize 100024ed f   MSVCRT:ucrt_stubs.obj
 0001:000014ed       ___scrt_stub_for_acrt_thread_attach 100024ed f   MSVCRT:ucrt_stubs.obj
 0001:000014ed       ___scrt_stub_for_acrt_thread_detach 100024ed f   MSVCRT:ucrt_stubs.obj
 0001:000014ed       ___scrt_stub_for_acrt_uninitialize 100024ed f   MSVCRT:ucrt_stubs.obj
 0001:000014ed       ___scrt_stub_for_acrt_uninitialize_critical 100024ed f   MSVCRT:ucrt_stubs.obj
 0001:000014ed       ___vcrt_initialize         100024ed f   MSVCRT:ucrt_stubs.obj
 0001:000014ed       ___vcrt_thread_attach      100024ed f   MSVCRT:ucrt_stubs.obj
 0001:000014ed       ___vcrt_thread_detach      100024ed f   MSVCRT:ucrt_stubs.obj
 0001:000014ed       ___vcrt_uninitialize       100024ed f   MSVCRT:ucrt_stubs.obj
 0001:000014ed       ___vcrt_uninitialize_critical 100024ed f   MSVCRT:ucrt_stubs.obj
 0001:000014f0       ___scrt_stub_for_is_c_termination_complete 100024f0 f   MSVCRT:ucrt_stubs.obj
 0001:000014f0       __is_c_termination_complete 100024f0 f   MSVCRT:ucrt_stubs.obj
 0001:000014f3       __filter_x86_sse2_floating_point_exception 100024f3 f   MSVCRT:x86_exception_filter.obj
 0001:000014f3       __filter_x86_sse2_floating_point_exception_default 100024f3 f   MSVCRT:x86_exception_filter.obj
 0002:00000000       __imp__InitializeSListHead@4 10003000     kernel32:KERNEL32.dll
 0002:00000004       __imp__IsDebuggerPresent@0 10003004     kernel32:KERNEL32.dll
 0002:00000008       __imp__DisableThreadLibraryCalls@4 10003008     kernel32:KERNEL32.dll
 0002:0000000c       __imp__GetSystemTimeAsFileTime@4 1000300c     kernel32:KERNEL32.dll
 0002:00000010       __imp__GetCurrentThreadId@0 10003010     kernel32:KERNEL32.dll
 0002:00000014       __imp__GetCurrentProcessId@0 10003014     kernel32:KERNEL32.dll
 0002:00000018       __imp__UnhandledExceptionFilter@4 10003018     kernel32:KERNEL32.dll
 0002:0000001c       __imp__SetUnhandledExceptionFilter@4 1000301c     kernel32:KERNEL32.dll
 0002:00000020       __imp__GetCurrentProcess@0 10003020     kernel32:KERNEL32.dll
 0002:00000024       __imp__TerminateProcess@8  10003024     kernel32:KERNEL32.dll
 0002:00000028       __imp__IsProcessorFeaturePresent@4 10003028     kernel32:KERNEL32.dll
 0002:0000002c       __imp__QueryPerformanceCounter@4 1000302c     kernel32:KERNEL32.dll
 0002:00000030       \177KERNEL32_NULL_THUNK_DATA 10003030     kernel32:KERNEL32.dll
 0002:00000034       __imp__memset              10003034     vcruntime:VCRUNTIME140.dll
 0002:00000038       __imp____std_type_info_destroy_list 10003038     vcruntime:VCRUNTIME140.dll
 0002:0000003c       __imp___except_handler4_common 1000303c     vcruntime:VCRUNTIME140.dll
 0002:00000040       \177VCRUNTIME140_NULL_THUNK_DATA 10003040     vcruntime:VCRUNTIME140.dll
 0002:00000044       __imp___execute_onexit_table 10003044     ucrt:api-ms-win-crt-runtime-l1-1-0.dll
 0002:00000048       __imp___configure_narrow_argv 10003048     ucrt:api-ms-win-crt-runtime-l1-1-0.dll
 0002:0000004c       __imp___cexit              1000304c     ucrt:api-ms-win-crt-runtime-l1-1-0.dll
 0002:00000050       __imp___initialize_onexit_table 10003050     ucrt:api-ms-win-crt-runtime-l1-1-0.dll
 0002:00000054       __imp___initterm           10003054     ucrt:api-ms-win-crt-runtime-l1-1-0.dll
 0002:00000058       __imp___initterm_e         10003058     ucrt:api-ms-win-crt-runtime-l1-1-0.dll
 0002:0000005c       __imp___seh_filter_dll     1000305c     ucrt:api-ms-win-crt-runtime-l1-1-0.dll
 0002:00000060       __imp___initialize_narrow_environment 10003060     ucrt:api-ms-win-crt-runtime-l1-1-0.dll
 0002:00000064       \177api-ms-win-crt-runtime-l1-1-0_NULL_THUNK_DATA 10003064     ucrt:api-ms-win-crt-runtime-l1-1-0.dll
 0002:00000068       __imp____stdio_common_vsprintf 10003068     ucrt:api-ms-win-crt-stdio-l1-1-0.dll
 0002:0000006c       \177api-ms-win-crt-stdio-l1-1-0_NULL_THUNK_DATA 1000306c     ucrt:api-ms-win-crt-stdio-l1-1-0.dll
 0002:00000070       __imp__JNU_ThrowInternalError@8 10003070     java:java.dll
 0002:00000074       \177java_NULL_THUNK_DATA   10003074     java:java.dll
 0002:00000078       __imp__JVM_GetManagement@4 10003078     jvm:jvm.dll
 0002:0000007c       __imp__JVM_GetVmArguments@4 1000307c     jvm:jvm.dll
 0002:00000080       __imp__JVM_ActiveProcessorCount@0 10003080     jvm:jvm.dll
 0002:00000084       __imp__JVM_GetAllThreads@8 10003084     jvm:jvm.dll
 0002:00000088       \177jvm_NULL_THUNK_DATA    10003088     jvm:jvm.dll
 0002:0000008c       ___guard_check_icall_fptr  1000308c     MSVCRT:guard_support.obj
 0002:00000090       ___castguard_check_failure_os_handled_fptr 10003090     MSVCRT:guard_support.obj
 0002:00000094       ___xc_a                    10003094     MSVCRT:initializers.obj
 0002:00000098       ___xc_z                    10003098     MSVCRT:initializers.obj
 0002:0000009c       ___xi_a                    1000309c     MSVCRT:initializers.obj
 0002:000000a0       ___xi_z                    100030a0     MSVCRT:initializers.obj
 0002:000000a4       ___xp_a                    100030a4     MSVCRT:initializers.obj
 0002:000000a8       ___xp_z                    100030a8     MSVCRT:initializers.obj
 0002:000000ac       ___xt_a                    100030ac     MSVCRT:initializers.obj
 0002:000000b0       ___xt_z                    100030b0     MSVCRT:initializers.obj
 0002:000000b8       ??_C@_0BJ@KKOPABNE@Memory?5Manager?5not?5found@ 100030b8     MemoryManagerImpl.obj
 0002:000000d4       ??_C@_0BG@EJKNNBCK@Memory?5Pool?5not?5found@ 100030d4     MemoryPoolImpl.obj
 0002:000000ec       ??_C@_05KBEOJPB@?$CFd?4?$CFd@ 100030ec     VMManagementImpl.obj
 0002:000000f4       ??_C@_01POHCFINO@Z@        100030f4     VMManagementImpl.obj
 0002:000000f8       ??_C@_0BK@DJAAMHIC@compTimeMonitoringSupport@ 100030f8     VMManagementImpl.obj
 0002:00000114       ??_C@_0CC@GDPMBOEP@threadContentionMonitoringSuppo@ 10003114     VMManagementImpl.obj
 0002:00000138       ??_C@_0BM@GCPPCNJD@currentThreadCpuTimeSupport@ 10003138     VMManagementImpl.obj
 0002:00000154       ??_C@_0BK@DMCEOMBH@otherThreadCpuTimeSupport@ 10003154     VMManagementImpl.obj
 0002:00000170       ??_C@_0BK@EJFDBCBP@objectMonitorUsageSupport@ 10003170     VMManagementImpl.obj
 0002:0000018c       ??_C@_0BJ@NIOHCHFH@synchronizerUsageSupport@ 1000318c     VMManagementImpl.obj
 0002:000001a8       ??_C@_0BN@GDBJIKMK@threadAllocatedMemorySupport@ 100031a8     VMManagementImpl.obj
 0002:000001c8       ??_C@_0CA@BBEOFMLC@remoteDiagnosticCommandsSupport@ 100031c8     VMManagementImpl.obj
 0002:000001e8       ??_C@_0BP@KJIDAONK@Unsupported?5Management?5version@ 100031e8     management.obj
 0002:00000208       __pDefaultRawDllMain       10003208     MSVCRT:dll_dllmain.obj
 0002:00000208       __pRawDllMain              10003208     MSVCRT:dll_dllmain.obj
 0002:00000218       __load_config_used         10003218     MSVCRT:loadcfg.obj
 0002:00000380       ___safe_se_handler_table   10003380     <linker-defined>
 0002:00000384       ___volatile_metadata       10003384     <linker-defined>
 0002:00000688       ___rtc_iaa                 10003688     MSVCRT:initsect.obj
 0002:0000068c       ___rtc_izz                 1000368c     MSVCRT:initsect.obj
 0002:00000690       ___rtc_taa                 10003690     MSVCRT:initsect.obj
 0002:00000694       ___rtc_tzz                 10003694     MSVCRT:initsect.obj
 0002:00001938       __IMPORT_DESCRIPTOR_jvm    10004938     jvm:jvm.dll
 0002:0000194c       __IMPORT_DESCRIPTOR_java   1000494c     java:java.dll
 0002:00001960       __IMPORT_DESCRIPTOR_KERNEL32 10004960     kernel32:KERNEL32.dll
 0002:00001974       __IMPORT_DESCRIPTOR_VCRUNTIME140 10004974     vcruntime:VCRUNTIME140.dll
 0002:00001988       __IMPORT_DESCRIPTOR_api-ms-win-crt-stdio-l1-1-0 10004988     ucrt:api-ms-win-crt-stdio-l1-1-0.dll
 0002:0000199c       __IMPORT_DESCRIPTOR_api-ms-win-crt-runtime-l1-1-0 1000499c     ucrt:api-ms-win-crt-runtime-l1-1-0.dll
 0002:000019b0       __NULL_IMPORT_DESCRIPTOR   100049b0     jvm:jvm.dll
 0003:00000000       ___security_cookie_complement 10005000     MSVCRT:gs_cookie.obj
 0003:00000004       ___security_cookie         10005004     MSVCRT:gs_cookie.obj
 0003:00000008       ___scrt_native_dllmain_reason 10005008     MSVCRT:utility.obj
 0003:00000010       ___isa_enabled             10005010     MSVCRT:cpu_disp.obj
 0003:00000014       ___scrt_ucrt_dll_is_in_use 10005014     MSVCRT:ucrt_stubs.obj
 0003:00000018       _jmm_interface             10005018     management.obj
 0003:0000001c       _jmm_version               1000501c     management.obj
 0003:00000020       _jvm                       10005020     management.obj
 0003:00000348       ?__type_info_root_node@@3U__type_info_node@@A 10005348     MSVCRT:tncleanup.obj
 0003:00000350       ?_OptionsStorage@?1??__local_stdio_scanf_options@@9@4_KA 10005350     MSVCRT:default_local_stdio_options.obj
 0003:00000358       ___scrt_current_native_startup_state 10005358     MSVCRT:utility.obj
 0003:0000035c       ___scrt_native_startup_lock 1000535c     MSVCRT:utility.obj
 0003:0000037c       ___scrt_debugger_hook_flag 1000537c     MSVCRT:utility_desktop.obj
 0003:00000380       ___isa_available           10005380     MSVCRT:cpu_disp.obj
 0003:00000384       ___favor                   10005384     MSVCRT:cpu_disp.obj
 0003:00000388       ?_OptionsStorage@?1??__local_stdio_printf_options@@9@9 10005388     <common>
 0003:00000390       ___dyn_tls_init_callback   10005390     <common>

 entry point at        0001:00000bb8

 Static symbols

 0000:ffff8000       .debug$S                   10000000     management.exp
 0000:ffff8000       .debug$S                   10000000     vcruntime:VCRUNTIME140.dll
 0000:ffff8000       .debug$S                   10000000     vcruntime:VCRUNTIME140.dll
 0000:ffff8000       .debug$S                   10000000     vcruntime:VCRUNTIME140.dll
 0000:ffff8000       .debug$S                   10000000     vcruntime:VCRUNTIME140.dll
 0000:ffff8000       .debug$S                   10000000     vcruntime:VCRUNTIME140.dll
 0000:ffff8000       .debug$S                   10000000     ucrt:api-ms-win-crt-runtime-l1-1-0.dll
 0000:ffff8000       .debug$S                   10000000     ucrt:api-ms-win-crt-runtime-l1-1-0.dll
 0000:ffff8000       .debug$S                   10000000     ucrt:api-ms-win-crt-runtime-l1-1-0.dll
 0000:ffff8000       .debug$S                   10000000     ucrt:api-ms-win-crt-runtime-l1-1-0.dll
 0000:ffff8000       .debug$S                   10000000     ucrt:api-ms-win-crt-runtime-l1-1-0.dll
 0000:ffff8000       .debug$S                   10000000     ucrt:api-ms-win-crt-runtime-l1-1-0.dll
 0000:ffff8000       .debug$S                   10000000     ucrt:api-ms-win-crt-runtime-l1-1-0.dll
 0000:ffff8000       .debug$S                   10000000     ucrt:api-ms-win-crt-runtime-l1-1-0.dll
 0000:ffff8000       .debug$S                   10000000     ucrt:api-ms-win-crt-runtime-l1-1-0.dll
 0000:ffff8000       .debug$S                   10000000     ucrt:api-ms-win-crt-runtime-l1-1-0.dll
 0000:ffff8000       .debug$S                   10000000     ucrt:api-ms-win-crt-runtime-l1-1-0.dll
 0000:ffff8000       .debug$S                   10000000     ucrt:api-ms-win-crt-runtime-l1-1-0.dll
 0000:ffff8000       .debug$S                   10000000     ucrt:api-ms-win-crt-runtime-l1-1-0.dll
 0000:ffff8000       .debug$S                   10000000     ucrt:api-ms-win-crt-stdio-l1-1-0.dll
 0000:ffff8000       .debug$S                   10000000     kernel32:KERNEL32.dll
 0000:ffff8000       .debug$S                   10000000     kernel32:KERNEL32.dll
 0000:ffff8000       .debug$S                   10000000     kernel32:KERNEL32.dll
 0000:ffff8000       .debug$S                   10000000     kernel32:KERNEL32.dll
 0000:ffff8000       .debug$S                   10000000     kernel32:KERNEL32.dll
 0000:ffff8000       .debug$S                   10000000     kernel32:KERNEL32.dll
 0000:ffff8000       .debug$S                   10000000     kernel32:KERNEL32.dll
 0000:ffff8000       .debug$S                   10000000     kernel32:KERNEL32.dll
 0000:ffff8000       .debug$S                   10000000     kernel32:KERNEL32.dll
 0000:ffff8000       .debug$S                   10000000     kernel32:KERNEL32.dll
 0000:ffff8000       .debug$S                   10000000     kernel32:KERNEL32.dll
 0000:ffff8000       .debug$S                   10000000     kernel32:KERNEL32.dll
 0000:ffff8000       .debug$S                   10000000     kernel32:KERNEL32.dll
 0000:ffff8000       .debug$S                   10000000     kernel32:KERNEL32.dll
 0000:ffff8000       .debug$S                   10000000     jvm:jvm.dll
 0000:ffff8000       .debug$S                   10000000     jvm:jvm.dll
 0000:ffff8000       .debug$S                   10000000     jvm:jvm.dll
 0000:ffff8000       .debug$S                   10000000     jvm:jvm.dll
 0000:ffff8000       .debug$S                   10000000     java:java.dll
 0001:00000770       _setStaticBooleanField     10001770 f   VMManagementImpl.obj
 0001:00000878       ?dllmain_crt_dispatch@@YGHQAUHINSTANCE__@@KQAX@Z 10001878 f   MSVCRT:dll_dllmain.obj
 0001:000008cb       ?dllmain_crt_process_attach@@YAHQAUHINSTANCE__@@QAX@Z 100018cb f   MSVCRT:dll_dllmain.obj
 0001:000009d2       ?dllmain_crt_process_detach@@YAH_N@Z 100019d2 f   MSVCRT:dll_dllmain.obj
 0001:00000a82       ?dllmain_dispatch@@YAHQAUHINSTANCE__@@KQAX@Z 10001a82 f   MSVCRT:dll_dllmain.obj
 0001:00000b8d       ?dllmain_raw@@YGHQAUHINSTANCE__@@KQAX@Z 10001b8d f   MSVCRT:dll_dllmain.obj
 0001:00000cfd       ___get_entropy             10001cfd f   MSVCRT:gs_support.obj
 0001:00000df2       ?find_pe_section@@YAPAU_IMAGE_SECTION_HEADER@@QAEI@Z 10001df2 f   MSVCRT:utility.obj
 0001:00001250       $$000000                   10002250     MSVCRT:sehprolg4.obj
 0002:0000020c       _GS_ExceptionPointers      1000320c     MSVCRT:gs_report.obj
 0002:00000698       __sehtable$?dllmain_crt_process_attach@@YAHQAUHINSTANCE__@@QAX@Z 10003698     MSVCRT:dll_dllmain.obj
 0002:000006b8       __sehtable$?dllmain_crt_process_detach@@YAH_N@Z 100036b8     MSVCRT:dll_dllmain.obj
 0002:000006e0       __sehtable$?dllmain_dispatch@@YAHQAUHINSTANCE__@@KQAX@Z 100036e0     MSVCRT:dll_dllmain.obj
 0002:00000700       __sehtable$___scrt_is_nonwritable_in_current_image 10003700     MSVCRT:utility.obj
 0002:00000720       .edata                     10003720     management.exp
 0002:00000748       rgpv                       10003748     management.exp
 0002:00000854       rgszName                   10003854     management.exp
 0002:00000960       rgwOrd                     10003960     management.exp
 0002:000009e6       szName                     100039e6     management.exp
 0002:000009f5       $N00001                    100039f5     management.exp
 0002:00000a03       $N00002                    10003a03     management.exp
 0002:00000a3c       $N00003                    10003a3c     management.exp
 0002:00000a7b       $N00004                    10003a7b     management.exp
 0002:00000ab9       $N00005                    10003ab9     management.exp
 0002:00000af5       $N00006                    10003af5     management.exp
 0002:00000b33       $N00007                    10003b33     management.exp
 0002:00000b68       $N00008                    10003b68     management.exp
 0002:00000b9a       $N00009                    10003b9a     management.exp
 0002:00000bcd       $N00010                    10003bcd     management.exp
 0002:00000bfd       $N00011                    10003bfd     management.exp
 0002:00000c36       $N00012                    10003c36     management.exp
 0002:00000c70       $N00013                    10003c70     management.exp
 0002:00000ca9       $N00014                    10003ca9     management.exp
 0002:00000cdd       $N00015                    10003cdd     management.exp
 0002:00000d0d       $N00016                    10003d0d     management.exp
 0002:00000d43       $N00017                    10003d43     management.exp
 0002:00000d82       $N00018                    10003d82     management.exp
 0002:00000dc1       $N00019                    10003dc1     management.exp
 0002:00000dfb       $N00020                    10003dfb     management.exp
 0002:00000e35       $N00021                    10003e35     management.exp
 0002:00000e65       $N00022                    10003e65     management.exp
 0002:00000e9e       $N00023                    10003e9e     management.exp
 0002:00000ede       $N00024                    10003ede     management.exp
 0002:00000f1b       $N00025                    10003f1b     management.exp
 0002:00000f58       $N00026                    10003f58     management.exp
 0002:00000f8a       $N00027                    10003f8a     management.exp
 0002:00000fc4       $N00028                    10003fc4     management.exp
 0002:00000ffe       $N00029                    10003ffe     management.exp
 0002:00001037       $N00030                    10004037     management.exp
 0002:00001070       $N00031                    10004070     management.exp
 0002:0000109d       $N00032                    1000409d     management.exp
 0002:000010dd       $N00033                    100040dd     management.exp
 0002:00001116       $N00034                    10004116     management.exp
 0002:0000114e       $N00035                    1000414e     management.exp
 0002:00001192       $N00036                    10004192     management.exp
 0002:000011db       $N00037                    100041db     management.exp
 0002:00001217       $N00038                    10004217     management.exp
 0002:00001256       $N00039                    10004256     management.exp
 0002:00001299       $N00040                    10004299     management.exp
 0002:000012d5       $N00041                    100042d5     management.exp
 0002:00001316       $N00042                    10004316     management.exp
 0002:00001353       $N00043                    10004353     management.exp
 0002:00001394       $N00044                    10004394     management.exp
 0002:000013cf       $N00045                    100043cf     management.exp
 0002:0000140a       $N00046                    1000440a     management.exp
 0002:00001444       $N00047                    10004444     management.exp
 0002:0000147f       $N00048                    1000447f     management.exp
 0002:000014b4       $N00049                    100044b4     management.exp
 0002:000014ee       $N00050                    100044ee     management.exp
 0002:0000152b       $N00051                    1000452b     management.exp
 0002:00001562       $N00052                    10004562     management.exp
 0002:000015ac       $N00053                    100045ac     management.exp
 0002:000015e7       $N00054                    100045e7     management.exp
 0002:00001623       $N00055                    10004623     management.exp
 0002:00001661       $N00056                    10004661     management.exp
 0002:0000169d       $N00057                    1000469d     management.exp
 0002:000016db       $N00058                    100046db     management.exp
 0002:00001718       $N00059                    10004718     management.exp
 0002:0000174b       $N00060                    1000474b     management.exp
 0002:00001783       $N00061                    10004783     management.exp
 0002:000017b8       $N00062                    100047b8     management.exp
 0002:000017ec       $N00063                    100047ec     management.exp
 0002:00001824       $N00064                    10004824     management.exp
 0002:00001866       $N00065                    10004866     management.exp
 0002:000018ad       $N00066                    100048ad     management.exp
 0002:000018f9       $N00067                    100048f9     management.exp
 0002:00001ab6       .idata$6                   10004ab6     jvm:jvm.dll
 0002:00001ada       .idata$6                   10004ada     java:java.dll
 0002:00001c08       .idata$6                   10004c08     kernel32:KERNEL32.dll
 0002:00001c5a       .idata$6                   10004c5a     vcruntime:VCRUNTIME140.dll
 0002:00001d2c       .idata$6                   10004d2c     ucrt:api-ms-win-crt-stdio-l1-1-0.dll
 0002:00001d4c       .idata$6                   10004d4c     ucrt:api-ms-win-crt-runtime-l1-1-0.dll
 0003:00000024       ?__proc_attached@@3HA      10005024     MSVCRT:dll_dllmain.obj
 0003:00000028       _GS_ExceptionRecord        10005028     MSVCRT:gs_report.obj
 0003:00000078       _GS_ContextRecord          10005078     MSVCRT:gs_report.obj
 0003:00000360       ?is_initialized_as_dll@@3_NA 10005360     MSVCRT:utility.obj
 0003:00000361       ?module_local_atexit_table_initialized@@3_NA 10005361     MSVCRT:utility.obj
 0003:00000364       ?module_local_atexit_table@@3U_onexit_table_t@@A 10005364     MSVCRT:utility.obj
 0003:00000370       ?module_local_at_quick_exit_table@@3U_onexit_table_t@@A 10005370     MSVCRT:utility.obj
 0004:00000060       $R000000                   10006060     management.dll.res
